:10000000F6282016201E2012A01A0A28A016432027
:10001000031831280830A9005720A80DA90B0C2877
:10002000201E3C2061205D20201A31203620280827
:100030000310F1282016201E2012201B2428FE3930
:10004000A50020170310F128A01B2C28AC00A01736
:100050004320031831282C084A2003183128201E79
:10006000F1283C2061202013A013A0122108840055
:10007000240884178004422821088400240980056C
:10008000841780050800362061203C205D2025086B
:10009000A01A0138A8000830A900A80D03183620BE
:1000A000031C3C2061205D20A90B4D2836206120D7
:1000B0002108840024080005FF3E2208840023094B
:1000C0003F28220884002308392883178001840AE6
:1000D000FF3E031D6628F1280830AC002518DA2001
:1000E0002208840023082519E920251DEB2021087A
:1000F000840024098417800521088400A70CA60C1D
:1001000000082404031C240680008920AC0B7C28F2
:10011000F1282208840023088006000080060800D9
:10012000A901A800FF30A807031CA907031CF12898
:100130000330A700DF309E209228A701E83EA600EA
:10014000A709FC30031CA728A6070318A428A607A4
:100150000000A70FA4282618AD28A61CB12800006F
:10016000B1280800A800A7010830AC00A60DA70D13
:1001700028082702031CBF282808A7020314A90D7A
:10018000AC0BB6282908F1281030AE00A701A60153
:10019000AD0CAC0C031CD2282808A60729080318AC
:1001A000290FA707A70CA60CAB0CAA0CAE0BC828EE
:1001B0002A08F128A801A901E128A70CA60CA80D7E
:1001C000A90DFF3E0318DD282908A7002808A6006E
:1001D000F1288004EE28FF3A8005EF28FF3A8417C3
:1001E000800583138312031300000800A001073069
:1001F0009F008316811320308400603083126620B4
:10020000A0308400503066202030840030306520DB
:10021000B6013330360203189E290630A100103093
:10022000A4000630A2000830A300D1301C20023008
:100230001C200120B9000630A1001030A4000630B7
:10024000A2000830A300D1301C2001301C20012066
:10025000B8000630A1001030A4000630A20008301B
:10026000A300D1301C2000301C200120B7007930C1
:10027000BE000530A1000430A4000530A200023009
:10028000A3000130A5003E08A6006C200630A600A1
:10029000A60B48294B290530A1000430A4000530E5
:1002A000A2000230A3000130A5003908A6006C208E
:1002B0000630A600A60B5A295D290530A10004309E
:1002C000A4000530A2000230A3000130A5003808C8
:1002D000A6006C200630A600A60B6C296F290530FD
:1002E000A1000430A4000530A2000230A3000130B8
:1002F000A5003708A6006C2083160510831205148C
:100300000630A600A60B82298529831605108312C4
:1003100005100130861B0301B1000130061B0301EB
:100320003104B1000130861A0301310403199929FF
:10033000BD22C8309020B60A031D0929B6010B3032
:1003400036020318342A0630A1001030A40006300B
:10035000A2000830A300D1301C2006301C20012050
:10036000BC000630A1001030A4000630A200083006
:10037000A300D1301C2005301C200120BB0006301A
:10038000A1001030A4000630A2000830A300D13034
:100390001C2004301C200120BA007A30BE00053039
:1003A000A1000430A4000530A2000230A3000130F7
:1003B000A5003E08A6006C200630A600A60BDE298C
:1003C000E1290530A1000430A4000530A20002306C
:1003D000A3000130A5003A08A6006C200630A60054
:1003E000A60BF029F3290530A1000430A400053044
:1003F000A2000230A3000130A5003B08A6006C203B
:100400000630A600A60B022A052A0530A1000430FA
:10041000A4000530A2000230A3000130A5003C0872
:10042000A6006C2083160510831205140630A60062
:10043000A60B182A1B2A83160510831205100130FB
:10044000861B0301B1000130061B03013104B1001A
:100450000130861A0301310403192F2AC423C8303E
:100460009020B60A031D9F29B6010B3036020318EF
:10047000BC2A0630A1001030A4000630A2000830CB
:10048000A30091301C200120BD003D08A6000A30C9
:10049000B220B300AD013308AC00A9010A30A800B6
:1004A000C420AF002B08B0002F083D02B400340870
:1004B000BD00BD17B31DBD133D17331D3D13BD1644
:1004C000B31CBD123D16331C3D122430BE00053056
:1004D000A1000430A4000530A2000230A3000130C6
:1004E000A5003E08A6006C200630A600A60B762AC2
:1004F000792A0530A1000430A4000530A2000230A2
:10050000A3000130A500FF30A6006C200630A60035
:10051000A60B882A8B2A0530A1000430A4000530E0
:10052000A2000230A3000130A5003D08A6006C2007
:100530000630A600A60B9A2A9D2A0530A100043099
:10054000A4000530A2000230A3000130A500FF3056
:10055000A6006C2083160510831205140630A60031
:10056000A60BB02AB32A8316051083120510C830D3
:100570009020B60A031D352A08290630A100103044
:10058000A4000630A2000830A300D1301C200230A5
:100590001C200120B9000630A1001030A400063054
:1005A000A2000830A300D1301C2001301C20012003
:1005B000B8000630A1001030A4000630A2000830B8
:1005C000A300D1301C2000301C200120B70079305E
:1005D000BE000530A1000430A4000530A2000230A6
:1005E000A3000130A5003E08A6006C200630A6003E
:1005F000A60BF82AFB2A0530A1000430A400053020
:10060000A2000230A3000130A5003908A6006C202A
:100610000630A600A60B0A2B0D2B0530A1000430D6
:10062000A4000530A2000230A3000130A500380864
:10063000A6006C200630A600A60B1C2B1F2B053035
:10064000A1000430A4000530A2000230A300013054
:10065000A5003708A6006C20831605108312051428
:100660000630A600A60B322B352B831605108312FD
:100670000510C8309020B20A861B442B3708B500FD
:1006800087233508B700B201061B4C2B3808B5008C
:1006900087233508B800B201861A542B3908B500F3
:1006A000A3233508B900B201FA3090200C30320291
:1006B000031D5B2B5C2BE92A0630A1001030A4003F
:1006C0000630A2000830A300D0301C2000301C20CF
:1006D00037081A200630A1001030A4000630A2000E
:1006E0000830A300D0301C2001301C2038081A200C
:1006F0000630A1001030A4000630A2000830A3008C
:10070000D0301C2002301C2039081A2008000F307D
:100710003505B30033083502B400340E0F39B40088
:10072000B30A0A303302031C9C2BB301B40A06300F
:100730003402031C9C2BB401340EF039B40033088E
:100740003407B50008000F303505B3003308350213
:10075000B400340E0F39B400B30A0A303302031C5C
:10076000B82BB301B40A06303402031CB82BB40111
:10077000340EF039B40033083407B50018303502B0
:10078000031CC32BB50108000630A1001030A400E3
:100790000630A2000830A300D1301C2006301C20F7
:1007A0000120BC000630A1001030A4000630A200D9
:1007B0000830A300D1301C2005301C200120BB00D4
:1007C0000630A1001030A4000630A2000830A300BB
:1007D000D1301C2004301C200120BA007A30BE0029
:1007E0000530A1000430A4000530A2000230A300AF
:1007F0000130A5003E08A6006C200630A600A60B1E
:10080000FF2B022C0530A1000430A4000530A2000B
:100810000230A3000130A5003A08A6006C20063083
:10082000A600A60B112C142C0530A1000430A40046
:100830000530A2000230A3000130A5003B08A6004D
:100840006C200630A600A60B232C262C0530A10018
:100850000430A4000530A2000230A3000130A5003E
:100860003C08A6006C208316051083120514063080
:10087000A600A60B392C3C2C8316051083120510FC
:10088000C8309020B20A861B4B2C3C08B5008E2441
:100890003508BC00B201061B532C3B08B500AA2446
:1008A0003508BB00B201861A5B2C3A08B500CC248F
:1008B0003508BA00B201FA3090200C303202031D24
:1008C000622C632CF02B0630A1001030A4000630FF
:1008D000A2000830A300D0301C2006301C203C08A9
:1008E0001A200630A1001030A4000630A200083003
:1008F000A300D0301C2005301C203B081A200630F5
:10090000A1001030A4000630A2000830A300D030AF
:100910001C2004301C203A081A2008000F3035052E
:10092000B30033083502B400340E0F39B400B30AF3
:100930000A303302031CA32CB301B40A0A30340278
:10094000031CA32CB401340EF039B400330834076F
:10095000B50008000F303505B30033083502B40088
:10096000340E0F39B400B30A0A303302031CBA2C18
:10097000B301B40A340EF039B40033083407B500BB
:1009800013303502031DC62C0130B500B508031D18
:10099000CB2C0130B50008000F303505B30033080B
:1009A0003502B400340E0F39B400B30A0A303302F2
:1009B000031CDC2CB301B40A340EF039B400330844
:1009C0003407B50032303502031DE82C0130B50084
:1009D000B508031DED2C0130B50008006300EE2CB6
:02400E00783FF9
:00000001FF
